:100000000C94280018950000189500001895000021
:10001000189500001895000018950000189500002C
:10002000189500000C94200C1895000018950000FD
:10003000189500001895000018950000189500000C
:1000400018950000189500001895000018950000FC
:100050008FE181BD87E181BD8FE58DBFC4E0E8E719
:100060004E2E88E08EBFD8E0F7E05F2EEEEFF7E08F
:10007000A0E6B0E088278D933197E9F783E389B94B
:1000800088E18AB9662487E08ABB87EF8BBB8FEB58
:1000900087BB8FEB88BB80EE84BB8FEF85BB80E88E
:1000A00081BB8BE382BB80E08FBD81E08EBD8FE1A1
:1000B00081BD87E181BD86E086B980E487B9C398B8
:1000C000C29AD89AC498C798C598F894A895709180
:1000D0006B007F7D70936B000027ABE6B0E08C91E6
:1000E00085FB0EF401E041E0041711F00C947C0054
:1000F00087E88ABB87E78BBB0E94660D7091D000B2
:1001000078607093D000EFEFF1E0A1ECB0E091E007
:100110000E9445280091C100003081E009F080E094
:100120008F930091C1000E3F80E010F009F081E054
:100130009F91892B882311F40C94A1008EEB80935E
:10014000C1000091C1004AE0040F01BF82E390E0CA
:100150000E940827ECEEF0E50E944F26ABE6B0E0E7
:100160008C9185FBA8E6B7E00E942D278D93882708
:100170008C930E9447260E945B26EAE0F0E0BB27B2
:10018000A0E10E9442280D3311F40C94FD00EBE035
:10019000F0E0A0E1BB2788E08C937BE70E94312848
:1001A000ECE0F0E001E010E0A0E1BB277BE70E947B
:1001B0003328EAE0F0E0A0E1BB278DE38C937BE7F6
:1001C0000E943128EEE0F0E0A0E1BB2780E08C93B4
:1001D0007BE70E943128E0E1F0E000E010E0A0E1E0
:1001E000BB277BE70E943328EFE0F0E0A0E1BB27CC
:1001F00080E08C937BE70E943128EBE0F0E0ACEBF1
:10020000B0E00E9442280091BC000C3318F011F0BD
:100210000C940C010C940F018CE38093BC0080E7DC
:1002200097E9ADEBB0E08D939C93ECE0F0E0A7EBA9
:10023000B0E00E944428EEE0F0E0A2ECB0E00E94C2
:100240004228EFE0F0E0A3ECB0E00E9442280E94D8
:100250006A0DE0E1F0E0A4E6B0E00E944428A4E6E4
:10026000B0E00E94CA25E0E1F0E0A4E6B0E07BE760
:100270000E943328A7EBB0E00D911C91003050E0B4
:10028000150711F00C944A0181E090E0A7EBB0E073
:100290008D939C93E4E0F1E50E944F26A8E6B7E039
:1002A000ECEBF0E00E949B270E944726ECE0F1E592
:1002B0000E944F26A8E6B7E0E7EBF0E00E948C270B
:1002C0000E944726ECE0F1E50E944F26A8E6B7E041
:1002D000E2ECF0E00E949B270E944726ECE0F1E56B
:1002E0000E944F26A8E6B7E0E3ECF0E00E949B27CF
:1002F0000E944726ECE0F1E50E944F26A8E6B7E011
:10030000E4E6F0E00E948C270E944726ECE0F1E54D
:100310000E944F26BB27A3E38C9180FBA8E6B7E0A1
:100320000E942D278D9388278C930E9447260E9438
:100330005B260027BB27A3E38C9180FB0EF401E032
:1003400041E0041711F00C94B10170916B007B7FB8
:1003500070936B00A2ECB0E08C918E7F8C930C9428
:10036000BB0170916B00746070936B00A2ECB0E005
:100370008C9181608C930027BB27A3E38C9183FB36
:100380000EF401E041E0041711F00C94D3017091D8
:10039000D0007F7D7093D000A2ECB0E08C918D7F77
:1003A0008C930C94DD017091D00070627093D0003A
:1003B000A2ECB0E08C9182608C9381E882BB80E0FB
:1003C0008093600081E08093620000916200083CAD
:1003D00018F011F00C940C020027BB27A0E38C91BD
:1003E00080FB0EF401E040E0041718F011F00C94CB
:1003F000FB010C940002A0E6B0E08C918F5F8C931F
:1004000081E090E00E940827A2E6B0E08C918F5F27
:100410008C9311F00C94E50100916000003011F014
:100420000C944802EEE0F1E50E944F260E945B2604
:1004300070916B007F7D70936B0070916B007064A6
:1004400070936B0081E08093620000916200043041
:1004500018F011F00C944602979A84E690E00E94FE
:100460000827979889E190E00E94082787E38ABBD4
:1004700087EC8BBB80E384BB8FEC85BBA2E6B0E04E
:100480008C918F5F8C9311F00C9425020C94560282
:10049000E8E1F1E50E944F260E945B2670916B0017
:1004A0007F7B70936B0080E882BB979880E080939D
:1004B000CF0070916B007D7F70936B0080E0809324
:1004C000C50086E08093BF008DE08093C00084E18A
:1004D00090E00E9408270E94F426C49AE2E2F1E527
:1004E0000E944F260E945B2688EC90E00E9408271D
:1004F000A89581B5886181BD877F81BDE0E6F0E088
:10050000FA93EA930E94471B2296A89500916000F7
:10051000003011F40C9498020E94891AECE2F1E583
:100520000E944F260E945B260E94300D0C949D0273
:100530007091D0007F7E7093D000E6E3F1E50E94D9
:100540004F260E94B21A84E690E00E9408270027F6
:10055000A0EDB0E08C9184FB0EF401E040E00417C4
:1005600011F00C94B5020E944A108FEF0E945E2693
:1005700082E390E00E9408277894A89581B588606E
:1005800081BDA3EBB0E04D915C91A7EBB0E00D9184
:100590001C910417150718F011F00C94D1020C945B
:1005A000D70281E090E0A7EBB0E08D939C93002709
:1005B000ABE6B0E08C9182FB0EF401E041E0041761
:1005C00081E009F080E08F930027A0EDB0E08C91EE
:1005D00084FB0EF401E040E0041781E009F080E0C4
:1005E0009F918923882311F40C940903E7EBF0E031
:1005F000FA93EA935A924A9280E0A42DB52D8C93F7
:1006000081E00E94B7250E941F0E249681E00E947F
:10061000B32580E08093B90080E080936A000027D2
:10062000A0EDB0E08C9184FB0EF401E041E00417F2
:1006300011F00C941D030E94660DA8950E943F26A0
:10064000ACE6B0E08D9388278C930091CF0000300A
:1006500081E009F080E08F930027BB27A3E38C9112
:1006600081FB0EF401E041E0041781E009F080E035
:100670009F91892B882311F40C945A030027ABE631
:10068000B0E08C9186FB0EF401E041E0041711F01C
:100690000C945303E3E6F0E0FA93EA930E945819AE
:1006A00022960C945A03E3E6F0E0FA93EA930E9450
:1006B0000D19229681E090E00E9408270091CF005A
:1006C000003081E009F080E08F930027ABE6B0E0D6
:1006D0008C9181FB0EF401E041E0041781E009F008
:1006E00080E09F91892B882311F40C947B0385E093
:1006F00090E00E940827ACE6B0E08C91803081E069
:1007000009F480E08F9300916300003081E009F4E8
:1007100080E09F91892B8F930091B900013081E097
:1007200009F080E09F91892B882311F40C940F032A
:1007300000916300003011F40C94D3050027BB270F
:10074000A3E38C9182FB0EF401E041E0041711F069
:100750000C943A048EB5887F8EBD8AE090E00E94AA
:1007600008270027ABE6B0E08C9186FB0EF401E091
:1007700041E0041711F00C94CE03E3E6F0E0FA93A5
:10078000EA930E9458192296A3E6B0E08C91A7EB59
:10079000B0E08D9388278C930C940704E3E6F0E097
:1007A000FA93EA930E940D1922960091630000309B
:1007B00011F40C940704A3E6B0E08C91A7EBB0E031
:1007C0008D9388278C9300916300043011F00C9472
:1007D000EF0383E090E0A7EBB0E08D939C93009152
:1007E0006300083011F00C94FB0384E090E0A7EB69
:1007F000B0E08D939C9300916300003111F00C9454
:10080000070485E090E0A7EBB0E08D939C93A3EB09
:10081000B0E04D915C91A7EBB0E00D911C910417F5
:10082000150780E010F009F081E08F93A7EBB0E0AE
:100830000D911C91003050E0150781E009F080E037
:100840009F91892B882311F40C942C0481E090E073
:10085000A7EBB0E08D939C9300916300003011F4FE
:100860000C943804ACE6B0E0E0E4F1E50E942E26FA
:100870000C94D3050027ABE6B0E08C9186FB0EF418
:1008800001E041E0041711F00C943F05E3E6F0E0CD
:10089000FA93EA930E9458192296009163000D3052
:1008A00011F00C945904ACE6B0E0E2E4F1E50E94EA
:1008B0002E26009163000F3011F00C94A104ABEDD3
:1008C000B0E00E94E527A4E6B0E00D931C93A3EBF3
:1008D000B0E04D915C91A4E6B0E00D911C9104173D
:1008E000150718F011F00C9477040C947D0481E046
:1008F00090E0A4E6B0E08D939C93A4E6B0E00D9167
:100900001C91003050E0150711F00C948F04ACE6F8
:10091000B0E0E4E4F1E50E942E260C949D04A4E6E8
:10092000B0E08D919C91A7EBB0E08D939C93ACE6E9
:10093000B0E0E0E4F1E50E942E26ABEDB0E08827C0
:100940008C9300916300013011F00C94AF04ABED77
:10095000B0E00E943426E6E4F1E50E942E260091E4
:100960006300023011F00C94BD04ABEDB0E00E94C6
:100970003426E8E4F1E50E942E260091630003305E
:1009800011F00C94CB04ABEDB0E00E943426EAE405
:10099000F1E50E942E2600916300053011F00C94C1
:1009A000D904ABEDB0E00E943426ECE4F1E50E94FE
:1009B0002E2600916300063011F00C94E704ABED95
:1009C000B0E00E943426EEE4F1E50E942E2600916C
:1009D0006300073011F00C94F504ABEDB0E00E9419
:1009E0003426E0E5F1E50E942E26009163000930EF
:1009F00011F00C940305ABEDB0E00E943426E2E563
:100A0000F1E50E942E26009163000A3011F00C944B
:100A10001105ABEDB0E00E943426E4E5F1E50E945B
:100A20002E26009163000B3011F00C941F05ABEDE6
:100A3000B0E00E943426E6E5F1E50E942E26009102
:100A400063000E3011F00C942D05ABEDB0E00E9468
:100A50003426E8E5F1E50E942E26ABEDB0E00E94D9
:100A60005C28082F033018F011F00C9439050C9411
:100A70003D05ABEDB0E088278C930C946A05E3E666
:100A8000F0E0FA93EA930E940D1922960091630018
:100A9000013011F00C945205ACE6B0E0E4E4F1E56D
:100AA0000E942E2600916300023011F00C945E0526
:100AB000ACE6B0E0EAE5F1E50E942E260091630085
:100AC000043011F00C946A05ACE6B0E0E2E4F1E524
:100AD0000E942E2600916300083011F00C94A005AE
:100AE0000091BC00033018F011F00C9479050C94BF
:100AF000A005ACEBB0E08C9183508C938EB5887FD1
:100B00008EBD5A924A928091BC00A42DB52D8C9333
:100B100081E00E94B7250E943522229681E00E9442
:100B2000B325EBE0F0E0ACEBB0E07BE70E943128CE
:100B30000091CF00013011F00C94A00581E08EBD32
:100B400000916300003111F00C94D3050091BC00BA
:100B5000063410F00C94D305ACEBB0E08C918D5FB3
:100B60008C938EB5887F8EBD5A924A928091BC003C
:100B7000A42DB52D8C9381E00E94B7250E943522CB
:100B8000229681E00E94B325EBE0F0E0ACEBB0E010
:100B90007BE70E9431280091CF00013011F00C94C6
:100BA000D30581E08EBDECE6F0E0ACE6B0E00E945B
:100BB00021270091B900013011F00C94000680E06B
:100BC0008093B900ACE6B0E0E4E4F1E50E942E26A3
:100BD0000027A0EDB0E08C9185FB0EF401E041E030
:100BE000041711F00C94000681E090E0A7EBB0E050
:100BF0008D939C93ACE6B0E0E0E4F1E50E942E26F4
:100C0000ACE6B0E0ECE5F1E50E94622811F00C944E
:100C100047065A924A928091BF00A42DB52D8C931D
:100C200081E00E94B7255A924A928091C000A42D7B
:100C3000B52D8C9381E00E94B7250E948E222496C8
:100C400082E00E94B3250091C30041E0042BA0E69E
:100C5000B0E00C937091D00074607093D0008EB5AA
:100C6000887F8EBDEFE0F0E0A0E6B0E07BE70E9479
:100C70003128809160008093C3000091CF00013043
:100C800011F00C94450681E08EBD0C94CA0BEEE584
:100C9000F1E50E94622811F00C948A065A924A9259
:100CA00080E0A42DB52D8C9381E00E94B7255A9247
:100CB0004A9280E0A42DB52D8C9381E00E94B72547
:100CC0000E948E22249682E00E94B3250091C300E8
:100CD0004EEF0423A0E6B0E00C937091D0007B7F30
:100CE0007093D0008EB5887F8EBDEFE0F0E0A0E677
:100CF000B0E07BE70E943128809160008093C300C0
:100D00000091CF00013011F00C94880681E08EBD77
:100D10000C94CA0BE0E4F1E50E94622811F00C94F7
:100D2000F5060091CF00013011F00C9499060E9455
:100D3000140DA3EBB0E04D915C91A7EBB0E00D91E9
:100D40001C910417150718F011F00C94F3060027F6
:100D5000A0EDB0E08C9184FB0EF401E040E00417BC
:100D600011F00C94C606E7EBF0E0FA93EA935A927E
:100D70004A9280E0A42DB52D8C9381E00E94B72586
:100D80000E941F0E249681E00E94B3250027A0ED4B
:100D9000B0E08C9184FB0EF401E041E0041711F007
:100DA0000C94F3060E94300D0027A0EDB0E08C916A
:100DB00084FB0EF401E040E0041711F00C94F306FC
:100DC000E7EBF0E0FA93EA935A924A9280E0A42D7E
:100DD000B52D8C9381E00E94B7250E941F0E2496AA
:100DE00081E00E94B3250C94CA0BE0E6F1E50E9475
:100DF000622811F00C9403070E94140D80E0809388
:100E0000C5000C94CA0BE2E4F1E50E94622811F0DF
:100E10000C943D070091CF00013011F00C943B077A
:100E20000027ABE6B0E08C9181FB0EF401E040E0DE
:100E3000041711F00C942D078EB5887F8EBD89B7ED
:100E40008B7F89BF70916B00726070936B0084E63A
:100E500090E00E9408270C943B0770916B007D7F07
:100E600070936B0080E29EE49DBD8CBD81E08EBDE1
:100E700089B7846089BF0C94CA0BE4E4F1E50E9451
:100E8000622811F00C94D5070091CF00013011F0C9
:100E90000C944C070E94140DA7EBB0E00E94CA25E9
:100EA0000027A0EDB0E08C9183FB0EF401E041E05F
:100EB000041711F00C9471070027ABE6B0E08C9199
:100EC00082FB0EF401E040E0041711F00C946C0773
:100ED000A7EBB0E00E94D0257091D000777F70938F
:100EE000D000A3EBB0E04D915C91A7EBB0E00D9189
:100EF0001C910417150718F011F00C9481070C943D
:100F0000870781E090E0A7EBB0E08D939C930027EA
:100F1000A0EDB0E08C9184FB0EF401E040E00417FA
:100F200011F00C94A607E7EBF0E0FA93EA935A92DB
:100F30004A9280E0A42DB52D8C9381E00E94B725C4
:100F40000E941F0E249681E00E94B3250027A0ED89
:100F5000B0E08C9184FB0EF401E041E0041711F045
:100F60000C94D3070E94300D0027A0EDB0E08C91C7
:100F700084FB0EF401E040E0041711F00C94D30759
:100F8000E7EBF0E0FA93EA935A924A9280E0A42DBC
:100F9000B52D8C9381E00E94B7250E941F0E2496E8
:100FA00081E00E94B3250C94CA0BEAE5F1E50E94AA
:100FB000622811F00C944D080091CF00013011F01F
:100FC0000C94E4070E94140DA7EBB0E00D911C9166
:100FD000013050E0150718F011F00C94F1070C9453
:100FE000F707A7EBB0E00E94D0250C94FF07A3EB16
:100FF000B0E08D919C91A7EBB0E08D939C9300277E
:10100000A0EDB0E08C9184FB0EF401E040E0041709
:1010100011F00C941E08E7EBF0E0FA93EA935A9271
:101020004A9280E0A42DB52D8C9381E00E94B725D3
:101030000E941F0E249681E00E94B3250027A0ED98
:10104000B0E08C9184FB0EF401E041E0041711F054
:101050000C944B080E94300D0027A0EDB0E08C915D
:1010600084FB0EF401E040E0041711F00C944B08EF
:10107000E7EBF0E0FA93EA935A924A9280E0A42DCB
:10108000B52D8C9381E00E94B7250E941F0E2496F7
:1010900081E00E94B3250C94CA0BE2E6F1E50E94C0
:1010A000622811F00C94C008A7EBB0E00E94CA259A
:1010B000A3EBB0E04D915C91A7EBB0E00D911C91DA
:1010C0000417150718F011F00C9468080C946E08BA
:1010D00081E090E0A7EBB0E08D939C938EB5887F84
:1010E0008EBDA3E7B0E00D911D912D913C91A3E938
:1010F000B0E00D931D932D933C930027A0EDB0E03D
:101100008C9184FB0EF401E040E0041711F00C9484
:10111000B6085A924A92A3E9B0E00D911D912D9123
:101120003C91A42DB52D0D931D932D933C9384E0FC
:101130000E94B7255A924A92A7EBB0E08D919C91FC
:10114000A42DB52D8D939C9382E00E94B7255A92D1
:101150004A9280E0A42DB52D8C9381E00E94B725A2
:101160000E945911269687E00E94B3250091CF0076
:10117000013011F00C94BE0881E08EBD0C94CA0BB6
:10118000E4E6F1E50E94622811F00C943409A7EB23
:10119000B0E00D911C91013050E0150718F011F0EE
:1011A0000C94D4080C94DA08A7EBB0E00E94D02588
:1011B0000C94E208A3EBB0E08D919C91A7EBB0E01A
:1011C0008D939C938EB5887F8EBDA3E7B0E00D9183
:1011D0001D912D913C91A3E9B0E00D931D932D93AA
:1011E0003C930027A0EDB0E08C9184FB0EF401E06D
:1011F00040E0041711F00C942A095A924A92A3E98C
:10120000B0E00D911D912D913C91A42DB52D0D9324
:101210001D932D933C9384E00E94B7255A924A92E5
:10122000A7EBB0E08D919C91A42DB52D8D939C934F
:1012300082E00E94B7255A924A9280E0A42DB52DF3
:101240008C9381E00E94B7250E945911269687E071
:101250000E94B3250091CF00013011F00C943209A7
:1012600081E08EBD0C94CA0BE6E6F1E50E9462288F
:1012700011F00C944409ECE0F0E0A7EBB0E07BE760
:101280000E9433280C94CA0BE8E6F1E50E9462281C
:1012900011F00C9458098DE181BD85E181BD0E945A
:1012A000140D81B5886081BD0C9454090C94CA0B4F
:1012B000ACE6B0E0EAE6F1E50E94622881E008F4DD
:1012C00080E08F93ACE6B0E0ECE6F1E50E946228A6
:1012D00081E010F009F080E09F918923882311F4C8
:1012E0000C942C0A89B78B7F89BF8EB5887F8EBD01
:1012F0000E943B26A0E6B0E08C9300916000003095
:1013000011F40C9478090E943F26A7EBB0E08D936E
:1013100088278C9380E08093CF0070916B007D7F55
:1013200070936B00A3EBB0E04D915C91A7EBB0E044
:101330000D911C910417150780E010F009F081E071
:101340008F93A7EBB0E00D911C91003050E0150792
:1013500081E009F080E09F91892B882311F40C949F
:10136000CC0981E090E0A7EBB0E08D939C93E7EB94
:10137000F0E0FA93EA935A924A9281E0A42DB52DB7
:101380008C9381E00E94B7250E941F0E249681E075
:101390000E94B3250C942A0A0027A0EDB0E08C919E
:1013A00084FB0EF401E040E0041781E009F080E0E6
:1013B0008F93ACE6B0E0EAE6F1E50E94622881E0B6
:1013C00009F080E09F918923882311F40C94FB0994
:1013D000E7EBF0E0FA93EA935A924A9281E0A42D67
:1013E000B52D8C9381E00E94B7250E941F0E249694
:1013F00081E00E94B3250027A0EDB0E08C9184FB32
:101400000EF401E040E0041781E009F080E08F93E2
:10141000ACE6B0E0ECE6F1E50E94622881E009F07C
:1014200080E09F918923882311F40C942A0AE7EB2A
:10143000F0E0FA93EA935A924A9280E0A42DB52DF7
:101440008C9381E00E94B7250E941F0E249681E0B4
:101450000E94B3250C94CA0BEEE6F1E50E946228C7
:1014600011F00C94670A0E943B26A0E6B0E08C9332
:1014700000916000003011F40C94330A0E943F2662
:10148000ACEBB0E08C938EB5887F8EBD5A924A92B9
:101490008091BC00A42DB52D8C9381E00E94B725CE
:1014A0000E943522229681E00E94B325EBE0F0E015
:1014B000ACEBB0E07BE70E9431280091CF00013017
:1014C00011F00C94650A81E08EBD0C94CA0BE0E724
:1014D000F1E50E94622811F00C94B50A0E943B26A7
:1014E000A0E6B0E08C9300916000003011F40C9401
:1014F0006E0A8091C200809360000E943F26A2EC99
:10150000B0E08C93A2ECB0E08C918F738C930E942E
:101510006A0D0091C20040E10423A0E6B0E00C9304
:1015200000916000003111F00C949A0A0E94660D3F
:101530000C949C0A0E94680DA2ECB0E08C918F7E06
:101540008C938EB5887F8EBDEEE0F0E0A2ECB0E02B
:101550007BE70E9431280091CF00013011F00C94FC
:10156000B30A81E08EBD0C94CA0BE2E7F1E50E945C
:10157000622811F00C94190B0091C2004FE3042370
:10158000A0E6B0E00C930091CF00013011F00C9474
:10159000CE0AA0E6B0E08C9180588C930027A0ED95
:1015A000B0E08C9184FB0EF401E041E0041711F0EF
:1015B0000C94DF0AA0E6B0E08C91805C8C9300274D
:1015C000ABE6B0E08C9181FB0EF401E041E0041742
:1015D00011F00C94F00AA0E6B0E08C91805E8C9340
:1015E0008091B700809362008EB5887F8EBD31E018
:1015F000A0E6B0E00E94562631E0ACEBB0E00E94DD
:10160000562631E0A2E6B0E00E9456268091B30053
:101610008093620031E0A2E6B0E00E94562600917D
:10162000CF00013011F00C94170B81E08EBD0C94AB
:10163000CA0BE4E7F1E50E94622811F00C949C0BC0
:10164000A6EDB0E00D911D912D913C91A2EDB0E081
:101650004D915D916D917C910E947427A6E6B0E05A
:101660000D931D932D933D93A6E6B0E00E94BB25FC
:10167000A6E6B0E00D911D912D913C9140E052E025
:1016800060E070E00E946826A6E6B0E00D931D932E
:101690002D933D93A6E6B0E00D911D912D913C91C7
:1016A000A4ECB0E04C915527662777270E946D2661
:1016B000A6E6B0E04D935D936D937D93A6E6B0E012
:1016C0000D911D912D913C914AE050E060E070E059
:1016D0000E946D26A6E6B0E04D935D936D937D93D9
:1016E00044E150E060E070E0A6E6B0E00D911D91AD
:1016F0002D913C910E9479270CF402C00C948A0B26
:1017000000E010E020E030E0A6E6B0E00D931D938D
:101710002D933C938EB5887F8EBD34E0A6E6B0E075
:101720000E9456260091CF00013011F00C949A0BC4
:1017300081E08EBD0C94CA0BE6E7F1E50E946228B9
:1017400011F00C94B40B8EB5887F8EBDA5EAB0E085
:101750000E9449260091CF00013011F00C94B20B89
:1017600081E08EBD0C94CA0BE8E7F1E50E94622887
:1017700011F00C94CA0B8EB5887F8EBD0E94F510B7
:101780000091CF00013011F00C94C80B81E08EBDA8
:101790000C94CA0B81E090E00E940827009163003E
:1017A000003011F40C941E0CA8950027ABE6B0E0B5
:1017B0008C9186FB0EF401E041E0041711F00C94CB
:1017C000EA0BE3E6F0E0FA93EA930E9458192296B6
:1017D0000C94F10BE3E6F0E0FA93EA930E940D1902
:1017E000229681E090E00E9408270091630000307B
:1017F00011F00C94D40B0091CF00013081E009F07E
:1018000080E08F930027ABE6B0E08C9181FB0EF473
:1018100001E041E0041781E009F080E09F91892B0D
:10182000882311F40C941A0C83E090E00E9408279E
:101830000C941E0C8AE090E00E9408270C940F0381
:101840000F921F922F923F924F925F927F928F92B0
:101850009F92AF92BF920F931F932F933F934F93FB
:101860005F936F937F938F939F93AF93BF93CF9328
:10187000DF93EF93FF938FB78F93F89489B78B7FA4
:1018800089BF8EB5887F8EBD5A924A9280E092E0E1
:10189000A42DB52D8D939C9382E00E94B7250E94C4
:1018A0003125229682E00E94B3250091DA000A30A9
:1018B00011F00C945D0C0E94660D0E947B1E00913D
:1018C000DA000A3011F00C946A0C0E94680D80E076
:1018D0008093DA00AAEDB0E08C918F5F8C93A8958D
:1018E0000027A0EDB0E08C9184FB0EF401E040E015
:1018F000041711F00C948F0C5A924A9280E092E0F7
:10190000A42DB52D8D939C9382E00E94B7250E9453
:101910003125229682E00E94B3250E947B1EA6ED0F
:10192000B0E04D915D916D917C91A2EDB0E00D9193
:101930001D912D913C910E94792780E00CF481E06B
:101940008F930027A0EDB0E08C9184FB0EF401E0B2
:1019500040E0041781E009F080E09F91892388230B
:1019600011F40C94BE0C80E49CE99DBD8CBD81E01B
:101970008EBD89B7846089BF0C94F40C80E080939D
:10198000CF0070916B007D7F70936B000027A0EDFE
:10199000B0E08C9184FB0EF401E040E0041711F0FC
:1019A0000C94DB0CABE6B0E08C9182FBA9EBB0E0D1
:1019B000882780F98C930091C2004FE70423A1E6A9
:1019C000B0E00C930E94680D80E08093C500002772
:1019D000ABE6B0E08C9185FB0EF401E041E004172A
:1019E00011F00C94F40CDF988F918FBFFF91EF9161
:1019F000DF91CF91BF91AF919F918F917F916F9127
:101A00005F914F913F912F911F910F91BF90AF9098
:101A10009F908F907F905F904F903F902F901F905E
:101A20000F901895F894FFCF89B78B7F89BF8EB53B
:101A3000887F8EBD80E08093CF0070916B007D7FAA
:101A400070936B000027ABE6B0E08C9185FB0EF441
:101A500001E041E0041711F00C942F0DDF98089578
:101A60006E98C498C598C7980E94680DE2E0F0E0AF
:101A70000E946226C49A0E94F42684E690E00E94A6
:101A80000827A8957091D0007F7E7093D000E0E683
:101A9000F0E0FA93EA930E94471B229600916000BF
:101AA000003011F40C94630D7091D000706170934C
:101AB000D00084E690E00E9408276E98C498C598EC
:101AC000C7980C94650D0E944A1008959798089540
:101AD000979A089581E00E94172770916B007B7F91
:101AE00070936B000091C20041E00423A881B9818A
:101AF0000C93A881B9810C91003011F40C94850DE0
:101B000070916B00746070936B007091D0007F7D5A
:101B10007093D0000091C20042E00423A881B981F3
:101B20000C93A881B9810C91003011F40C949D0D97
:101B30007091D00070627093D0007091D0007F7B64
:101B40007093D0000091C20044E00423A881B981C1
:101B50000C93A881B9810C91003011F40C94B50D4F
:101B60007091D00070647093D0007091D0007F7736
:101B70007093D0000091C20048E00423A881B9818D
:101B80000C93A881B9810C91003011F40C94CD0D07
:101B90007091D00070687093D00070916B00777F67
:101BA00070936B000091C20040E20423A881B981C8
:101BB0000C93A881B9810C91003011F40C94E50DBF
:101BC00070916B00786070936B007091D0007B7F98
:101BD0007093D0000091C30041E00423A881B98133
:101BE0000C93A881B9810C91003011F40C94FD0D77
:101BF0007091D00074607093D0000091C30046E0F3
:101C00000423A881B9810C93A881B9810C9142E089
:101C10000E944C280C93A881B9818C918093D100AB
:101C20000091D100033011F00C94190E82E08093E2
:101C3000D10081E0481A8827580A2296089582E048
:101C40000E94172781E00E9417278EB5887F8EBDDE
:101C500070916B007D7F70936B00A3E7B0E00D91F6
:101C60001D912D913C91A3E9B0E00D931D932D930F
:101C70003C935A924A92A3E9B0E00D911D912D91A7
:101C80003C91A42DB52D0D931D932D933C9384E091
:101C90000E94B7255A924A92AA85BB858D919C9144
:101CA000A42DB52D8D939C9382E00E94B7255A9266
:101CB0004A9280E0A42DB52D8C9381E00E94B72537
:101CC0000E945911269687E00E94B32540E050E01B
:101CD00060E070E0AFE8B0E00D911D912D913C9176
:101CE0000E94792711F00C94770E0C9444100E94F6
:101CF000E9215A924A928091BC00A42DB52D8C9373
:101D000081E00E94B7250E943522229681E00E9440
:101D1000B3255A924A92ADEBB0E08D919C91A42DDF
:101D2000B52D8D939C9382E00E94B7250E94CD2211
:101D3000229682E00E94B3250027A0EDB0E08C91AE
:101D400082FB0EF401E041E0041711F00C94C20E86
:101D50005A924A928091BF00A42DB52D8C9381E0B8
:101D60000E94B7255A924A928091C000A42DB52DA9
:101D70008C9381E00E94B7250E948E22249682E0F7
:101D80000E94B325A3E9B0E00D911D912D913C91E6
:101D9000A2EDB0E00D931D932D933C93A3E9B0E029
:101DA0000D911D912D913C91AFE8B0E04D915D9169
:101DB0006D917C910E946F27A6EDB0E00D931D936D
:101DC0002D933D9380E0A881B9818C930E947B1E66
:101DD00081E090E0AA81BB818D939C93AA81BB8115
:101DE0000D911C910F3F51E0150718F011F00C9464
:101DF000280FAA81BB81AD90BC90AFEDB0E0AA0DD9
:101E0000BB1D0C910F3F81E009F080E08F93AA8108
:101E1000BB81AD90BC90A0EEB0E0AA0DBB1D0C91B3
:101E20000F3E80E010F009F081E09F918923882324
:101E300011F40C94210F81E0A881B9818C930C944A
:101E4000280FAA81BB810E94CA2511F00C94EE0EC6
:101E5000A881B9810C91013011F00C94E60EAA8191
:101E6000BB81AD90BC90A1EEB0E0AA0DBB1D8C91E2
:101E7000AA81BB818D9388278C93AA81BB810D9108
:101E80001C9140E150E00E94E825AA81BB814D935E
:101E90005C9380E18093C400AA81BB810D911C9169
:101EA000013050E0150711F00C945B0F84E0809333
:101EB000C4000C94E80F023050E0150711F00C94A8
:101EC000660F85E08093C4000C94E80F033050E067
:101ED000150711F00C94710F86E08093C4000C94E8
:101EE000E80F043050E0150711F00C947C0F87E0E8
:101EF0008093C4000C94E80F053050E0150711F0F2
:101F00000C94870F88E08093C4000C94E80F06308F
:101F100050E0150711F00C94920F8AE08093C400F2
:101F20000C94E80F073050E0150711F00C949D0F4A
:101F30008CE08093C4000C94E80F083050E0150743
:101F400011F00C94A80F8EE08093C4000C94E80F5D
:101F5000093050E0150711F00C94B30F80E1809325
:101F6000C4000C94E80F0A3050E0150711F00C94EF
:101F7000BE0F84E18093C4000C94E80F0B3050E056
:101F8000150711F00C94C90F88E18093C4000C94DC
:101F9000E80F0C3050E0150711F00C94D40F8CE1D1
:101FA0008093C4000C94E80F0D3050E0150711F039
:101FB0000C94DF0F80E28093C4000C94E80F0E3085
:101FC00050E0150711F00C94E80F88E28093C400EC
:101FD000AFE8B0E00D911D912D913C9140E052E0B1
:101FE00060E070E00E946826A6E6B0E00D931D93C5
:101FF0002D933D93A6E6B0E00D911D912D913C915E
:10200000A4ECB0E04C915527662777270E946D26F7
:10201000A6E6B0E04D935D936D937D93A6E6B0E0A8
:102020000D911D912D913C9148EE53E060E070E0E0
:102030000E946D26A6E6B0E04D935D936D937D936F
:10204000AC81BD810C91003011F00C94441000273C
:10205000ABE6B0E08C9185FB0EF401E041E00417A3
:1020600011F00C943410DF9A81E08093CF0088EC5B
:102070009FEA9DBD8CBD89B7846089BF81E08EBD1C
:1020800085E090E00E94082783E0481A8827580AD4
:1020900024960895A895A3E7B0E00D911D912D9188
:1020A0003C91A7E7B0E00D931D932D933C93A3E7DC
:1020B000B0E00D911D912D913C91A3E9B0E00D93FD
:1020C0001D932D933C935A924A92A3E9B0E00D914F
:1020D0001D912D913C91A42DB52D0D931D932D9304
:1020E0003C9384E00E94B7255A924A9280E090E0A7
:1020F000A42DB52D8D939C9382E00E94B7255A9212
:102100004A9280E0A42DB52D8C9381E00E94B725E2
:102110000E945911269687E00E94B325A895A3EB4B
:10212000B0E00D911C91013050E0150710F00C94B7
:10213000C0105A924A9281E0A42DB52D8C9381E073
:102140000E94B7250E942723229681E00E94B32592
:102150008CE291E00E9408275A924A9280E0A42DD6
:10216000B52D8C9381E00E94B7250E9427232296EB
:1021700081E00E94B3257091D00070617093D0000F
:10218000A895A3E7B0E00D911D912D913C91A3E995
:10219000B0E00D931D932D933C93A7EBB0E00D9110
:1021A0001C91003050E0150781E009F080E08F932A
:1021B000A3EBB0E04D915C91A7EBB0E00D911C91C9
:1021C0000417150780E010F009F081E09F91892B3A
:1021D000882311F40C94F21081E090E0A7EBB0E0BA
:1021E0008D939C930E94680D089584E00E941727A8
:1021F000A2EDB0E00D911D912D913C91A881B98186
:102200000D931D932D933C93A3E7B0E00D911D9189
:102210002D913C91A3E9B0E00D931D932D933C9338
:102220005A924A92A3E9B0E00D911D912D913C91F3
:10223000A42DB52D0D931D932D933C9384E00E9406
:10224000B7255A924A928FE19EE4A42DB52D8D9325
:102250009C9382E00E94B7255A924A9280E0A42D76
:10226000B52D8C9381E00E94B7250E9459112696C6
:1022700087E00E94B325A3E7B0E00D911D912D9159
:102280003C91A3E9B0E00D931D932D933C93A8815D
:10229000B9810D911D912D913C91A2EDB0E00D936E
:1022A0001D932D933C9384E0481A8827580A229660
:1022B000089581E00E94172781E00E94172781E09E
:1022C0000E94172780E090E0A5EBB0E08D939C93EF
:1022D00070916B007F7E70936B0000E010E020E057
:1022E00030E0AFE8B0E00D931D932D933C930027B1
:1022F000ABE6B0E08C9183FB0EF401E041E0041703
:1023000081E009F080E08F93A885B9850D911C913B
:10231000003050E0150781E009F480E09F918923A7
:102320008F93AE81BF810C91003081E009F080E095
:102330009F918923882311F40C94F911A7E9B0E047
:10234000E885F9850E948C27E7E9F0E0A8E6B7E088
:102350000E941728E8E6F7E0A7E9B0E01127222756
:1023600004E033270E94312781E4AC81BD818C9346
:10237000AC81BD818C9180939D0081E0E7E9F0E024
:1023800001E00A93ACE6B0E00E941C28ACE6B0E0A5
:102390008C91AEE9B0E08C9382E0E7E9F0E001E0F7
:1023A0000A93ACE6B0E00E941C28ACE6B0E08C9149
:1023B000AFE9B0E08C9383E0E7E9F0E001E00A9355
:1023C000ACE6B0E00E941C28ACE6B0E08C91A0EA3C
:1023D000B0E08C9384E0E7E9F0E001E00A93ACE63A
:1023E000B0E00E941C28ACE6B0E08C91A1EAB0E01D
:1023F0008C9389B78B7F89BF8EB5887F8EBD81B561
:10240000886181BD877F81BDABECB0E00D911D91EE
:102410002D913C91A7ECB0E00D931D932D933C932F
:10242000A7E7B0E04D915D916D917C91A3E7B0E09D
:102430000D911D912D913C910E94792711F00C94E2
:102440002B1202E010E020E030E0A7ECB0E00D93AA
:102450001D932D933C9380E0A881B9818C93EA81F0
:10246000FB81FA93EA935A924A92AE85BF850D9109
:102470001D912D913C91A42DB52D0D931D932D9360
:102480003C9384E00E94B7250E947220249684E049
:102490000E94B325AA81BB810C910E3F11F40C94CC
:1024A0005D127091D00070617093D00070916B00DC
:1024B000706170936B000C9470125A924A92AA85C4
:1024C000BB858D919C91A42DB52D8D939C9382E01D
:1024D0000E94B7250E947113229682E00E94B325C4
:1024E000A881B9818C918F5F8C9340917000A881F5
:1024F000B9810C91041781E009F080E08F930027E7
:10250000ABE6B0E08C9184FB0EF401E041E00417EF
:1025100081E009F480E09F918923882311F40C94D1
:10252000261300917F000B3011F00C94D312E7ECCE
:10253000F0E0FA93EA935A924A92A7ECB0E00D9138
:102540001D912D913C91A42DB52D0D931D932D938F
:102550003C9384E00E94B7250E94B117249684E042
:102560000E94B325EA85FB85FA93EA935A924A9230
:10257000A7ECB0E00D911D912D913C91A42DB52DAE
:102580000D931D932D933C9384E00E94B7250E94E8
:102590004717249684E00E94B32580E0A881B98182
:1025A0008C930C942413A7E7B0E04D915D916D914D
:1025B0007C91A3E7B0E00D911D912D913C910E947B
:1025C000792711F00C94EA12AA85BB850E94BB25DD
:1025D0000C942413E7ECF0E0FA93EA935A924A92AF
:1025E000A7ECB0E00D911D912D913C91A42DB52D3E
:1025F0000D931D932D933C9384E00E94B7250E9478
:10260000B117249684E00E94B325EA85FB85FA93EE
:10261000EA935A924A92A7ECB0E00D911D912D9148
:102620003C91A42DB52D0D931D932D933C9384E0E7
:102630000E94B7250E944717249684E00E94B32584
:1026400080E0A881B9818C930C942A13AA85BB855C
:102650000E94BB250027ABE6B0E08C9184FB0EF412
:1026600001E041E0041711F00C942F12C49AA885E0
:10267000B9850D911C91003050E0150711F00C94B4
:102680004913A5EBB0E08D919C91A3EBB0E08D9345
:102690009C930091CF00013081E009F080E08F939E
:1026A0000027A0EDB0E08C9184FB0EF401E040E047
:1026B000041781E009F080E09F918923882311F4B9
:1026C0000C946B1380E593EC9DBD8CBD81E08EBDB9
:1026D00089B7846089BF83E0481A8827580A2696FC
:1026E000089584E00E94172784E00E94172781E064
:1026F0000E94172781E00E94172781E00E94172778
:1027000081E00E94172780E0AE81BF818C93AE816B
:10271000BF810C910F3018F011F00C94541581E02A
:10272000AC81BD818C93AC81BD810C910C3018F0D3
:1027300011F00C94B3138FEF0E94FB260E94FD262C
:102740000E94FC26AC81BD81AD90BB24A1E8B0E025
:10275000AA0DBB1D8C93AC81BD818C918F5F8C9336
:1027600011F00C9493138DE0AC81BD818C93AC81FE
:10277000BD810C91043118F011F00C94D1138FEF3E
:102780000E94FB260E94FD260E94FC26A881B9819A
:102790008C93AC81BD818C918F5F8C9311F00C94E4
:1027A000B713EA85FB85FA93EA93EA85FB85FA93EA
:1027B000EA930E94DC1524960027ABE6B0E08C91EA
:1027C00084FB0EF401E041E0041711F00C94EA13CD
:1027D0000C944C1580E0AA81BB818C9300918D00F4
:1027E000003281E009F080E08F9300918D0000318C
:1027F00081E009F080E09F91892B882311F40C94EB
:10280000051481E0AA81BB818C9300918200003085
:1028100081E009F480E08F9300918200053E81E021
:1028200009F480E09F9189238F93AA81BB810C9149
:10283000013081E009F080E09F918923882311F421
:102840000C94411500918D00003211F00C942C1461
:10285000A5EBB0E00E94CA250027ABE6B0E08C9162
:1028600083FB0EF401E040E0041711F00C946114B6
:1028700081E0AC81BD818C93AC85BD854D915C912F
:10288000A5EBB0E00D911C910417150781E009F04C
:1028900080E08F93A5EBB0E00D911C91003050E0EB
:1028A000150780E010F009F081E09F9189238823CB
:1028B00011F40C945F1480E0AC81BD818C930C9476
:1028C000951480E0AC81BD818C9381E0A881B981B1
:1028D0008C93A881B9810C91053018F011F00C94FB
:1028E0009514A881B981AD90BB24ACE9B0E0AA0DE4
:1028F000BB1D4C91A881B981AD90BB24A1E8B0E08B
:10290000AA0DBB1D0C91041711F40C948D1481E0D9
:10291000AC81BD818C930C949514A881B9818C9164
:102920008F5F8C9311F00C946914AC81BD810C9174
:10293000003081E009F080E08F93AC85BD850D917A
:102940001C910F315EE4150781E009F080E09F9152
:10295000892B882311F40C9441150E946E15A885CB
:10296000B9850D911D912D913C9140E052E060E0C0
:1029700070E00E946D26AFE8B0E04D935D936D93DB
:102980007D93E3E9F0E0FA93EA935A924A92AE8596
:10299000BF850D911D912D913C91A42DB52D0D93C9
:1029A0001D932D933C9384E00E94B7250E94471706
:1029B000249684E00E94B32580918D0080938E0040
:1029C000AC85BD850D911C910F315EE4150711F0AA
:1029D0000C941215A8E6B7E0E5EBF0E00E948C2716
:1029E0000E944726EAE7F1E50E944F26A5EAB0E0FB
:1029F0000E944926EAE7F1E50E944F2600918D00EA
:102A0000003111F00C940815ECE7F1E50E944F2617
:102A1000A8E6B7E0E885F9850E948F270E9447263F
:102A20000E945B26AC81BD810C91003011F00C94AA
:102A3000411570916B00706170936B0000918E0076
:102A4000003181E009F080E08F93AC85BD850D9168
:102A50001C910F315EE4150781E009F480E09F913D
:102A60008923882311F40C944115AA85BB850D9107
:102A70001D912D913C91ABECB0E00D931D932D93E6
:102A80003C9300918200003011F00C944C15709131
:102A90006B00706170936B00AE81BF818C918F5F12
:102AA0008C9311F00C9487138FEF0E94FB260E94E9
:102AB000FD260E94FC26A0E6B0E08C938FEF0E94DA
:102AC000FB260E94FD260E94FC26A0E6B0E08C9327
:102AD0008CE0481A8827580A2C96089581E00E94B5
:102AE0001727A5EAB0E088278C9381E0A881B981F7
:102AF0008C93A881B9810C91083018F011F00C94D6
:102B0000A815A881B981AD90BB24A1E8B0E0AA0DB9
:102B1000BB1D0C91003211F40C94A015A881B98151
:102B2000AD90BB24A1E8B0E0AA0DBB1D8C91A5EA35
:102B3000B0E08F930E9434268F918D9388278C93D9
:102B4000A881B9818C918F5F8C9311F00C947915C9
:102B5000A5EAB0E00E943426E0E8F1E50E942E26C6
:102B600089E0A881B9818C93A881B9810C910B303F
:102B700018F011F00C94D615A881B981AD90BB2442
:102B8000A1E8B0E0AA0DBB1D8C91A5EAB0E08F933F
:102B90000E9434268F918D9388278C93A881B981C8
:102BA0008C918F5F8C9311F00C94B41581E0481ACE
:102BB0008827580A2296089581E00E94172781E00D
:102BC0000E94172784E00E9417278FEF0E94FB26A0
:102BD0000E94FD260E94FC26AC81BD818C938FEF64
:102BE0000E94FB260E94FD260E94FC26AA81BB8132
:102BF0008C93AA81BB810C9111272227332740E0B7
:102C000051E060E070E00E946826A885B9850D93C8
:102C10001D932D933D93A885B9850D911D912D91FF
:102C20003C91AC81BD814C915527662777270E9446
:102C30006F27A885B9850D931D932D933D93A88586
:102C4000B9850D911D912D913C9140E050E061E0DE
:102C500070E00E946826A881B9810D931D932D9381
:102C60003D938FEF0E94FB260E94FD260E94FC26CA
:102C7000AC81BD818C938FEF0E94FB260E94FD26C4
:102C80000E94FC26AC81BD818C938FEF0E94FB26B5
:102C90000E94FD260E94FC26AC81BD818C938FEFA3
:102CA0000E94FB260E94FD260E94FC26AC81BD816D
:102CB0008C938FEF0E94FB260E94FD260E94FC262B
:102CC000AC81BD818C938FEF0E94FB260E94FD2674
:102CD0000E94FC26AA81BB818C93AA81BB810C91A6
:102CE00011272227332740E051E060E070E00E9486
:102CF0006826A885B9850D931D932D933D93A885CE
:102D0000B9850D911D912D913C91AC81BD814C9166
:102D10005527662777270E946F27A885B9850D93C9
:102D20001D932D933D93A885B9850D911D912D91EE
:102D30003C91A881B9814D915D916D917C910E94EA
:102D40006F27A885B9850D931D932D933D938FEF24
:102D50000E94FB260E94FD260E94FC26AC81BD81BC
:102D60008C938FEF0E94FB260E94FD260E94FC267A
:102D7000AA81BB818C93AA81BB810C911127222748
:102D8000332740E051E060E070E00E946826A881AF
:102D9000B9810D931D932D933D93A881B9810D9118
:102DA0001D912D913C91AC81BD814C915527662799
:102DB00077270E946F27A881B9810D931D932D93CA
:102DC0003D938FEF0E94FB260E94FD260E94FC2669
:102DD000AC81BD818C938FEF0E94FB260E94FD2663
:102DE0000E94FC26AA81BB818C93AA81BB810C9195
:102DF00011272227332740E051E060E070E00E9475
:102E00006826AE81BF810D931D932D933D93AE81B6
:102E1000BF810D911D912D913C91AC81BD814C9153
:102E20005527662777270E946F27AE81BF810D93B4
:102E30001D932D933D93AE81BF810D911D912D91D9
:102E40003C9140E050E061E070E00E946826AE8175
:102E5000BF810D931D932D933D93AE81BF810D9145
:102E60001D912D913C91A881B9814D915D916D91FC
:102E70007C910E946F27AE81BF810D931D932D938E
:102E80003D9386E0481A8827580A2696089584E0DC
:102E90000E94172784E00E941727AC81BD810D9105
:102EA0001D912D913C9142E050E060E070E00E9465
:102EB0007427A881B9810D931D932D933D93A0E7AD
:102EC000B0E00C91112722273327A881B9814D91B9
:102ED0005D916D917C910E946826AA81BB810D93C2
:102EE0001D932D933D93AA81BB810D911D912D9131
:102EF0003C91A7E7B0E04D915D916D917C910E946E
:102F00006F27AA81BB810D931D932D933D93009153
:102F10007F000B3011F40C949F17AA81BB810D9197
:102F20001D912D913C9140E250E060E070E00E94E4
:102F30006F27AA81BB810D931D932D933D93AA8189
:102F4000BB810D911D912D913C91AE81BF810D935F
:102F50001D932D933C9388E0481A8827580A24969D
:102F6000089584E00E94172782E00E9417270091AD
:102F70007F000B3011F00C94F517AC81BD810D91E1
:102F80001D912D913C9140E850E060E070E00E947E
:102F90006D26A2EDB0E04D935D936D937D93AC8172
:102FA000BD810D911C9140E850E00E940826A88147
:102FB000B9810D931C93A881B9810D911C9144E0B6
:102FC00050E00E942226A881B9810D931C93A8810C
:102FD000B9810D911C9144E050E0040F151FA881A8
:102FE000B9810D931C930C942B18AC81BD810D916C
:102FF0001D912D913C9140E051E060E070E00E9415
:103000006D26A2EDB0E04D935D936D937D93AC8101
:10301000BD810D911C9140E051E00E940826A881DD
:10302000B9810D931C93A881B9810D911C9142E047
:1030300050E00E942226A881B9810D931C93A8819B
:10304000B9810D911C9142E050E0040F151FA88139
:10305000B9810D931C93A2EDB0E00D911D912D91BE
:103060003C91ABE7B0E04D915D916D917C910E94F8
:103070006F27A2EDB0E00D931D932D933D93A2ED2C
:10308000B0E00D911D912D913C91AEE6B0E04D91D7
:103090005C91662777270E946F27A2EDB0E00D9321
:1030A0001D932D933D930E947B1EA881B981AD9005
:1030B000BC90AFEDB0E0AA0DBB1D8C91AA81BB8185
:1030C0008D9388278D938D938C93A881B9810E94CD
:1030D000D025AA81BB810D911D912D913C9140E09D
:1030E00051E060E070E00E946826AA81BB810D93E8
:1030F0001D932D933D93AA81BB810D911D912D911F
:103100003C91A881B981AD90BC90AFEDB0E0AA0D23
:10311000BB1D4C915527662777270E946F27AA81F0
:10312000BB810D931D932D933D9300917F000B3038
:1031300011F00C94FB18A881B9810E94D025AA81B6
:10314000BB810D911D912D913C9140E051E060E0DB
:1031500070E00E946826AA81BB810D931D932D9378
:103160003D93AA81BB810D911D912D913C91A88128
:10317000B981AD90BC90AFEDB0E0AA0DBB1D4C91F4
:103180005527662777270E946F27AA81BB810D9359
:103190001D932D933D93A881B9810E94D025AA81CA
:1031A000BB810D911D912D913C9140E051E060E07B
:1031B00070E00E946826AA81BB810D931D932D9318
:1031C0003D93AA81BB810D911D912D913C91A881C8
:1031D000B981AD90BC90AFEDB0E0AA0DBB1D4C9194
:1031E0005527662777270E946F27AA81BB810D93F9
:1031F0001D932D933D93AA81BB810D911D912D911E
:103200003C91AE81BF810D931D932D933C9386E03D
:10321000481A8827580A2496089581E00E941727A3
:1032200081E00E94172709B340EF0423AA81BB81E4
:103230000C93AA81BB810C9148E00E944C280C930E
:103240000027BB27A3E38C9184FB0EF401E041E04F
:10325000041711F00C943119AA81BB818C918F5FF6
:103260008C93AA81BB818C9180958C93AA81BB8120
:103270000C914FE10423AC81BD810C930027ABE698
:10328000B0E08C9185FB0EF401E041E0041711F0F1
:103290000C945219AA81BB810C914FE00423AC819C
:1032A000BD810C9382E0481A8827580A2496089515
:1032B00081E00E941727DF9AAF9ADE9AAE9ADD9AD4
:1032C000AD9ADC9AAC9A80E0AA81BB818C93AD98D0
:1032D000E881F981FA93EA930E94F3192296AD9A54
:1032E000A881B9810C91003018F011F00C947A1972
:1032F0000C948419A881B9810C9144E0049FAA819F
:10330000BB810C920C94ED19DD98E881F981FA9358
:10331000EA930E94F3192296DD9AA881B9810C9153
:10332000003018F011F00C9497190C94A719A8818B
:10333000B9810C9144E0049F0C92A881B9810C9151
:1033400041E0041BAA81BB810C930C94ED19AC984D
:10335000E881F981FA93EA930E94F3192296AC9AD4
:10336000A881B9810C91003018F011F00C94BA19B1
:103370000C94CA19A881B9810C9144E0049F0C9265
:10338000A881B9810C9142E0041BAA81BB810C93F6
:103390000C94ED19DC98E881F981FA93EA930E9484
:1033A000F3192296DC9AA881B9810C91003018F0AB
:1033B00011F00C94DD190C94ED19A881B9810C91D0
:1033C00044E0049F0C92A881B9810C9143E0041B56
:1033D000AA81BB810C930C94ED1981E0481A8827CF
:1033E000580A2296089581E00E94172781E00E94E2
:1033F0001727AA81BB8189B38C93AA81BB818C9149
:1034000080958C93AA81BB810C9140E40E944C284A
:103410000C93AA81BB810C91003011F00C94321AEC
:10342000A881B98183B38C93A881B9818C9180954F
:103430008C93A881B9810C9140E40E944C280C9394
:10344000A881B9810C91003018F011F00C942A1A5F
:103450000C94321AA881B9810C9142E0040FAA8120
:10346000BB810C93AA81BB810C91033011F00C94A9
:103470003F1A82E0AA81BB818C930C944A1AAA81DC
:10348000BB810C91023011F00C944A1A83E0AA819E
:10349000BB818C93AA81BB818C91AC81BD818C93C3
:1034A00082E0481A8827580A2496089581E00E94ED
:1034B000172781E0A881B9818C93AA81BB814C91A7
:1034C000A881B9810C91041718F011F00C94831A9B
:1034D0005A924A9282E0A42DB52D8C9381E00E94ED
:1034E000B7250E942723229681E00E94B3258DE70D
:1034F00090E00E940827A881B9818C918F5F8C93FE
:1035000011F00C945D1A81E0481A8827580A229617
:10351000089581E00E94172781E0A881B9818C93EA
:10352000A881B9810C91063018F011F00C94AC1AF6
:103530000E94660D8FE090E00E9408270E94680DAF
:1035400084E690E00E940827A881B9818C918F5F62
:103550008C9311F00C94901A81E0481A8827580A2D
:10356000229608950E94F426C39A80E991E00E9471
:10357000082781B5886081BD0E94E9215A924A924C
:1035800081E0A42DB52D8C9381E00E94B7250E9487
:103590003522229681E00E94B32581B5886181BDE4
:1035A000877F81BD88EC90E00E940827FF27E0E13B
:1035B000FA93EA935A924A928BE0A42DB52D8C93FC
:1035C00081E00E94B7250E94BD24249681E00E94DC
:1035D000B325013051E0150711F00C94081B5A92E5
:1035E0004A92ADEBB0E08D919C91A42DB52D8D93B9
:1035F0009C9382E00E94B7250E94CD22229682E011
:103600000E94B325E2E8F1E50E944F260E945B2666
:103610005A924A9282E3A42DB52D8C9381E00E94A8
:10362000B7250E943522229681E00E94B325C29AD6
:10363000D89A82E390E00E940827089581E00E94D2
:10364000172781E00E9417278FEFAA81BB818C93F7
:1036500080E0A881B9818C93A881B9810C91073051
:1036600018F011F00C94411B91E0AA81BB810E94DB
:10367000EA26A881B9818C918F5F8C9311F00C940C
:103680002C1B82E0481A8827580A2496089581E066
:103690000E94172781E00E94172781E00E941727C8
:1036A00082E00E94172782E00E9417278FEFAA85E9
:1036B000BB858C9381E0A885B9858C93A885B98555
:1036C0000C91003418F011F00C94701B0E941E1B1A
:1036D000A885B9858C918F5F8C9311F00C945E1B3B
:1036E000C49881E0A885B9858C93A885B9850C918B
:1036F000003418F011F00C94871B0E941E1BA88543
:10370000B9858C918F5F8C9311F00C94751B8AE0B6
:1037100090E00E940827A895EE81FF81FA93EA9332
:103720005A924A9280E4A42DB52D8C9381E00E9498
:10373000B7255A924A9200E010E020E030E0A42D34
:10374000B52D0D931D932D933C9384E00E94B725D6
:103750000E945821269685E00E94B325AE81BF8144
:103760000C91013011F40C94BE1BC49AE6E8F1E50B
:103770000E944F260E945B260C94751E81E0AA854C
:10378000BB858C93A89580E090E0A881B9818D934A
:103790009C93EE81FF81FA93EA935A924A9281E4D4
:1037A000A42DB52D8C9381E00E94B7255A924A92A0
:1037B00000E010E020E030E0A42DB52D0D931D9326
:1037C0002D933C9384E00E94B7250E9458212696B1
:1037D00085E00E94B325A881B9810E94CA25AE81E7
:1037E000BF810C91003081E009F080E08F93A881C7
:1037F000B9810D911C91003050E0150781E009F06E
:1038000080E09F91892B882311F40C94C91BC49AE2
:10381000A881B9810D911C91003050E0150711F07D
:103820000C941A1CEEE8F1E50E944F260E945B26DC
:103830000C94751EA89584E690E00E940827A89530
:10384000C49881E090E00E940827EE81FF81FA93FE
:10385000EA935A924A9280E5A42DB52D8C9381E08B
:103860000E94B7255A924A9201E010E020E030E031
:10387000A42DB52D0D931D932D933C9384E00E94B0
:10388000B7250E945821269685E00E94B32585E041
:1038900090E00E940827C49A8AE090E00E940827DE
:1038A000A89500E010E020E030E0ABE7B0E00D9339
:1038B0001D932D933C9300E010E020E030E0A2ED5A
:1038C000B0E00D931D932D933C930E947B1E00E06E
:1038D00010E020E030E0A2EDB0E00D931D932D93B9
:1038E0003C930027A0EDB0E08C9184FB0EF401E046
:1038F00041E0041711F00C947F1C0C94751EA895E0
:103900000091EC00023011F40C94131D8091A2027E
:1039100080937F00A9EAB2E00D91112740E051E0C9
:103920000E942226AA81BB810D931C93AA81BB8190
:103930000D911C91A8EAB2E04D915527040F151F77
:10394000AA81BB810D931C93AA81BB810D911C910F
:103950002227332740E050E061E070E00E946826B3
:10396000ABE7B0E00D931D932D933D93A7EAB2E032
:103970000D91112740E051E00E942226AA81BB81CF
:103980000D931C93AA81BB810D911C91A6EAB2E014
:103990004D915527040F151FAA81BB810D931C93D0
:1039A000ABE7B0E00D911D912D913C91AA81BB81B7
:1039B0004D915C91662777270E946F27ABE7B0E0B7
:1039C0000D931D932D933D9300917F000C3011F0CA
:1039D0000C94ED1C8BE080937F0000917F000E30F3
:1039E00011F00C94F61C8BE080937F0000917F0017
:1039F0000F3011F00C94FF1C8BE080937F00ABE73D
:103A0000B0E00D911D912D913C91A2EDB0E00D9390
:103A10001D932D933C930E947B1EA2EDB0E00E946B
:103A2000D6250C94671D00911601063411F00C94F4
:103A30003D1D84E080937F0087E3A885B9858C9342
:103A4000A885B9850C910C3318F011F00C943B1D2E
:103A5000A885B985AD90BB24AFEDB0E0AA0DBB1D24
:103A60008C910E945E26A885B9858C918F5F8C937E
:103A700011F00C94201D0E945B2600913201063447
:103A800011F00C94671D8BE080937F0083E5A8857F
:103A9000B9858C93A885B9850C91073518F011F07C
:103AA0000C94651DA885B985AD90BB24AFEDB0E041
:103AB000AA0DBB1D8C910E945E26A885B9858C91AC
:103AC0008F5F8C9311F00C944A1D0E945B26E8E9ED
:103AD000F1E50E944F26A8E6B7E0EFE7F0E00E948C
:103AE0009B270E9447260E945B26EAEAF1E50E9496
:103AF0004F26A8E6B7E0EBE7F0E00E948F270E9490
:103B000047260E945B2684E0A885B9858C93A8850A
:103B1000B9850C910B3018F011F00C94A21DA885FA
:103B2000B985AD90BB24AFEDB0E0AA0DBB1D8C9163
:103B30000E945E26A885B9858C918F5F8C9311F0C9
:103B40000C94871D0E945B268091ED00809370008D
:103B5000ECEBF1E50E944F26A8E6B7E0E0E7F0E0E5
:103B60000E949B270E9447260E945B2600917000BE
:103B7000003011F00C94BE1D0C94751E0091700065
:103B8000003418F011F00C94C71D0C94C91D0C944E
:103B9000751E8091EE00AE81BF818C938091EF0005
:103BA000AC81BD818C93AC81BD819C91AE81BF8184
:103BB0008C91AEE6B0E08D939C938091F600AE813F
:103BC000BF818C938091F700AC81BD818C93AC81D7
:103BD000BD819C91AE81BF818C91A1E7B0E08D93B6
:103BE0009C93A1E7B0E00D911C91003050E01507C7
:103BF00011F00C94111E80910401AE81BF818C9351
:103C000080910501AC81BD818C93AC81BD819C917B
:103C1000AE81BF818C91A1E7B0E08D939C930C9411
:103C2000111EA1E7B0E00D911C91003050E0150786
:103C300011F00C941D1E0C94751E02E010E020E0A3
:103C400030E0A1E7B0E04D915C91662777270E94B4
:103C50006826A3E7B0E00D931D932D933D93A3E752
:103C6000B0E00D911D912D913C91AEE6B0E04D91EB
:103C70005C91662777270E946F27A3E7B0E00D933A
:103C80001D932D933D93A3E7B0E00D911D912D91D0
:103C90003C91A2EDB0E04D915D916D917C910E94BF
:103CA0006F27A3E7B0E00D931D932D933D93ECECAC
:103CB000F1E50E944F26A8E6B7E0E3E7F0E00E94B6
:103CC0008F270E9447260E945B26A3E7B0E00D9154
:103CD0001D912D913C91A2EDB0E00D931D932D937C
:103CE0003C9380E0AA85BB858C9387E0481A88279F
:103CF000580A2A96089581E00E94172781E00E94C1
:103D0000172782E00E94172782E00E9417278FEF73
:103D1000AE81BF818C9391E0AE81BF810E94EA2683
:103D200091E0AE81BF810E94EA2691E0AE81BF8121
:103D30000E94EA2691E0AE81BF810E94EA2691E0CE
:103D4000AE81BF810E94EA2691E0AE81BF810E94D0
:103D5000EA2691E0AE81BF810E94EA2691E0AE8121
:103D6000BF810E94EA2691E0AE81BF810E94EA26CF
:103D700091E0AE81BF810E94EA2691E0AE81BF81D1
:103D80000E94EA2691E0AE81BF810E94EA2691E07E
:103D9000AE81BF810E94EA2691E0AE81BF810E9480
:103DA000EA2691E0AE81BF810E94EA2691E0AE81D1
:103DB000BF810E94EA26C49880E090E0A881B98182
:103DC0008D939C938FEF0E94FB260E94FD260E94FC
:103DD000FC26AE81BF818C93A881B9810E94CA253F
:103DE000AE81BF810C91003081E009F480E08F93B7
:103DF000A881B9810D911C91003050E0150781E038
:103E000009F080E09F91892B882311F40C94E21E25
:103E1000A881B9810D911C91003050E0150711F077
:103E20000C941F1FE4EDF1E50E944F260E945B26D3
:103E30007091D00070617093D0000C946C20EE8172
:103E4000FF81FA93EA935A924A9281E5A42DB52D07
:103E50008C9381E00E94B7255A924A92A2EDB0E07D
:103E60000D911D912D913C91A42DB52D0D931D9378
:103E70002D933C9384E00E94B7250E9458212696FA
:103E800085E00E94B3250027A0EDB0E08C9184FB73
:103E90000EF401E041E0041711F00C945F1FE2EE14
:103EA000F1E50E944F26A8E6B7E0E2EDF0E00E94BF
:103EB0008F270E9447260E945B260C946C20A895B1
:103EC000AE81BF810C91003011F00C94AA1F80E0EC
:103ED00090E0A881B9818D939C938FEF0E94FB267F
:103EE0000E94FD260E94FC26AE81BF818C93A88192
:103EF000B9810E94CA25AE81BF810C91003081E05A
:103F000009F480E08F93A881B9810D911C91003054
:103F100050E0150781E009F080E09F91892B88230C
:103F200011F40C946D1FA881B9810D911C91003082
:103F300050E0150711F00C94AA1FECEFF1E50E9478
:103F40004F260E945B267091D00070617093D00064
:103F50000C946C20AE81BF810C910F3F11F00C943A
:103F6000F41F80E090E0A881B9818D939C938FEF3E
:103F70000E94FB260E94FD260E94FC26AE81BF8186
:103F80008C93A881B9810E94CA25AE81BF810C9112
:103F90000F3F81E009F480E08F93A881B9810D91F2
:103FA0001C91003050E0150781E009F080E09F91FE
:103FB000892B882311F40C94B71FA881B9810D9126
:103FC0001C91003050E0150711F00C94F41FEAE04A
:103FD000F2E50E944F260E945B267091D00070612E
:103FE0007093D0000C946C20AE81BF810C910E3F79
:103FF00011F40C941120E8E1F2E50E944F26A8E6A6
:10400000B7E0EE81FF810E949B270E9447260E9415
:104010005B26C49A7091D00070617093D0000C94AC
:104020006C2080E090E0AA81BB818D939C9380E01E
:10403000AE81BF818C93AE81BF810C910F3F18F090
:1040400011F00C945320AA81BB810E94CA258FEFE6
:104050000E94FB260E94FD260E94FC26AA81BB81AD
:10406000AD90BC90AFEDB0E0AA0DBB1D8C93AA81C2
:10407000BB810E94CA258FEF0E94FB260E94FD266D
:104080000E94FC26AA81BB81AD90BC90AFEDB0E050
:10409000AA0DBB1D8C93AE81BF818C918F5F8C93D9
:1040A00011F00C941B208FEF0E94FB260E94FD262E
:1040B0000E94FC26AE81BF818C938FEF0E94FB266D
:1040C0000E94FD260E94FC26AE81BF818C93C49A7B
:1040D000A2EDB0E00E94BB2586E0481A8827580A66
:1040E0002896089582E00E94172781E00E941727F2
:1040F00080E0AE81BF818C930E941E1BC49880E03B
:1041000090E0AA81BB818D939C938FEF0E94FB2648
:104110000E94FD260E94FC26A881B9818C93AA8169
:10412000BB810E94CA25A881B9810C91003081E031
:1041300009F480E08F93AA81BB810D911C9100301E
:1041400050E0150781E009F080E09F91892B8823DA
:1041500011F40C948520AA81BB810D911C91003033
:1041600050E0150711F00C94C220E4EDF1E50E9437
:104170004F260E945B267091D00070617093D00032
:104180000C945221E881F981FA93EA935A924A9267
:1041900081E5A42DB52D8C9381E00E94B7255A921C
:1041A0004A92AA85BB850D911D912D913C91A42D1C
:1041B000B52D0D931D932D933C9384E00E94B7255C
:1041C0000E945821269685E00E94B325A881B981D6
:1041D0000C91003011F00C94192180E090E0AA813C
:1041E000BB818D939C938FEF0E94FB260E94FD263E
:1041F0000E94FC26A881B9818C93AA81BB810E9470
:10420000CA25A881B9810C91003081E009F480E0D1
:104210008F93AA81BB810D911C91003050E015074E
:1042200081E009F080E09F91892B882311F40C94A0
:10423000F320A881B9810C910F3F11F00C944C210F
:1042400080E090E0AA81BB818D939C938FEF0E94C8
:10425000FB260E94FD260E94FC26A881B9818C9332
:10426000AA81BB810E94CA25A881B9810C910F3F08
:1042700081E009F480E08F93AA81BB810D911C91AC
:10428000003050E0150781E009F080E09F91892B14
:10429000882311F40C942621A881B9818C91AE81D8
:1042A000BF818C9383E0481A8827580A2496089582
:1042B00084E00E94172781E00E94172782E00E9475
:1042C00017278FEFAA81BB818C9391E0AA81BB81D4
:1042D0000E94EA2691E0A885B9850E94EA26AE816F
:1042E000BF810D911D912D913C9140E052E060E025
:1042F00070E00E946826AC81BD810D931D932D93C3
:104300003D93AC81BD818F9314968E910E94DE21E6
:104310008E910E94DE218E910E94DE218E910E945C
:10432000DE2185E90E94DE218F9180E090E0A88166
:10433000B9818D939C938FEF0E94FB260E94FD26EE
:104340000E94FC26AA81BB818C93A881B9810E941E
:10435000CA25AA81BB810C910F3F81E009F480E05E
:104360008F93A881B9810D911C91003050E0150701
:1043700081E009F080E09F91892B882311F40C944F
:104380009B21A881B9810D911C91003050E0150747
:1043900011F00C94D621E6E2F2E50E944F260E942D
:1043A0005B267091D00070617093D000AA81BB81B0
:1043B0008C91AA85BB858C930C94E3218FB9779B54
:1043C000FECF8FB1089587E0481A8827580A2696AD
:1043D00008955A924A9284E298E0A42DB52D8D93C7
:1043E0009C9382E00E94B7255A924A9280E0A42DC5
:1043F000B52D8C9381E00E94B7250E9462242496FB
:1044000083E00E94B325EF93FF93ECE8F1E00E9474
:10441000DC26FF91EF91BB27A0E38C9182FBDEF7B6
:1044200089E190E00E9408275A924A9280E298E03F
:10443000A42DB52D8D939C9382E00E94B7255A92AE
:104440004A9280E0A42DB52D8C9381E00E94B7257F
:104450000E946224249683E00E94B32589E190E0C3
:104460000E9408270E94EA22089582E00E941727EE
:1044700000E011E0AA81BB814D9155270E942226C0
:10448000A881B9810D931C93A881B9810D911C91CC
:10449000AA81BB814D915527040F151FA881B981B1
:1044A0000D931C935A924A92AA81BB818D919C9143
:1044B000A42DB52D8D939C9382E00E94B7255A922E
:1044C0004A928BE0A42DB52D8C9381E00E94B725F4
:1044D0000E946224249683E00E94B3255A924A9255
:1044E00080E298E0A42DB52D8D939C9382E00E94EC
:1044F000B7255A924A9280E0A42DB52D8C9381E085
:104500000E94B7250E946224249683E00E94B3256E
:1045100082E0481A8827580A2296089582E00E946D
:10452000172700E110E0AC81BD814D9155270E9415
:104530002226A881B9810D931C93A881B9810D9180
:104540001C91AA81BB814D915527040F151FA8818D
:10455000B9810D931C935A924A92AA81BB818D9185
:104560009C91A42DB52D8D939C9382E00E94B7253C
:104570005A924A9282E0A42DB52D8C9381E00E943C
:10458000B7250E946224249683E00E94B32582E02E
:10459000481A8827580A229608955A924A92AA8160
:1045A000BB818D919C91A42DB52D8D939C9382E020
:1045B0000E94B7255A924A9283E0A42DB52D8C9380
:1045C00081E00E94B7250E946224249683E00E9425
:1045D000B325089581E00E94172781E00E941727E4
:1045E000C49AD898C29880E0A881B9818C9380E061
:1045F000AA81BB818C93AA81BB810C910F3118F0E9
:1046000011F00C941F2391E0A881B9810E94EA2641
:1046100091E0A881B9810E94EA2691E0A881B98140
:104620000E94EA2691E0A881B9810E94EA26AA8127
:10463000BB818C918F5F8C9311F00C94FB22C29AFA
:10464000D89A82E0481A8827580A2496089581E06B
:104650000E9417275A924A9280E298E0A42DB52D25
:104660008D939C9382E00E94B7255A924A9280E0F3
:10467000A42DB52D8C9381E00E94B7250E94622461
:10468000249683E00E94B325AA81BB810C9100305F
:1046900011F00C945A235A924A9280E0A42DB52D21
:1046A0008C9381E00E94B7250E94D423229681E05A
:1046B0000E94B325AA81BB810C91013011F00C94AA
:1046C00070235A924A9285E6A42DB52D8C9381E0F1
:1046D0000E94B7250E94D423229681E00E94B32530
:1046E000AA81BB810C91023011F00C949D235A9247
:1046F0004A9283E6A42DB52D8C9381E00E94B725C4
:104700000E94D423229681E00E94B32588EC90E099
:104710000E9408275A924A9280E0A42DB52D8C93CE
:1047200081E00E94B7250E94D423229681E00E9456
:10473000B32582E390E00E940827AA81BB810C91F7
:10474000033011F00C94C6235A924A9282E6A42DAB
:10475000B52D8C9381E00E94B7250E94D423229628
:1047600081E00E94B32580E991E00E9408275A92D7
:104770004A9280E0A42DB52D8C9381E00E94B7254C
:104780000E94D423229681E00E94B3258AE090E023
:104790000E9408278AE090E00E94082781E0481ADA
:1047A0008827580A2296089581E00E941727C49A04
:1047B000D898C298AA81BB810C91003018F011F0F2
:1047C0000C94E4230C941E2483E5A881B9818C9376
:1047D00091E0A881B9810E94EA268FEEA881B98173
:1047E0008C9391E0A881B9810E94EA268EE6A88187
:1047F000B9818C9391E0A881B9810E94EA2691E069
:10480000AA81BB810E94EA2680E0A881B9818C93AD
:1048100091E0A881B9810E94EA2691E0A881B9813E
:104820000E94EA2691E0A881B9810E94EA2691E0DF
:10483000A881B9810E94EA260C945A2485E4A881B3
:10484000B9818C9391E0A881B9810E94EA2688E71A
:10485000A881B9818C9391E0A881B9810E94EA2650
:1048600089E6A881B9818C9391E0A881B9810E94E1
:10487000EA2684E7A881B9818C9391E0A881B98167
:104880000E94EA2680E0A881B9818C9391E0A881FA
:10489000B9810E94EA2691E0A881B9810E94EA26A6
:1048A00091E0A881B9810E94EA2691E0A881B981AE
:1048B0000E94EA26C29AD89A81E0481A8827580AA4
:1048C0002296089581E00E941727C29AD8985A929A
:1048D0004A9282E0A42DB52D8C9381E00E94B725E9
:1048E0000E941725229681E00E94B3255A924A928F
:1048F000AC81BD818C91A42DB52D8C9381E00E945B
:10490000B7250E941725229681E00E94B325AC812D
:10491000BD8111968C91A881B9818C935A924A924B
:10492000AA81BB818C91A42DB52D8C9381E00E942E
:10493000B7250E941725229681E00E94B325AC81FD
:10494000BD818C91A881B9818C935A924A92AA8197
:10495000BB818C91A42DB52D8C9381E00E94B7254D
:104960000E941725229681E00E94B325D89A81E003
:10497000481A8827580A2296089581E00E9417272E
:1049800081E00E94172782E00E941727C29AD898D8
:104990005A924A9283E0A42DB52D8C9381E00E9417
:1049A000B7250E941725229681E00E94B3255A92CE
:1049B0004A92A885B9858C91A42DB52D8C9381E060
:1049C0000E94B7250E941725229681E00E94B325F8
:1049D000EC81FD81FA93EA930E941D252296EA81DB
:1049E000FB81FA93EA930E941D252296D89AAC8106
:1049F000BD810D91112740E051E00E942226A8813F
:104A0000B9810D931C93A881B9810D911C91AA8144
:104A1000BB814D915527040F151FA885B9850D93AE
:104A20001C9384E0481A8827580A2696089591E036
:104A3000A881B9810E94EA26089581E00E94172783
:104A400091E0A881B9810E94DF26A881B9818C916B
:104A5000AA81BB818C9381E0481A8827580A229644
:104A6000089582E00E94172781E00E941727C49AC8
:104A7000BB27A0E38C9182FBDEF7C298AC81BD819D
:104A80000D911C91003052E0150711F00C94802517
:104A900081E090E0AA81BB818D939C9380E0A88106
:104AA000B9818C93A881B9810C910F3018F011F065
:104AB0000C947E25BB27A0E38C9182FBDEF790E26D
:104AC000AA81BB81AD90BC90AFEDB0E0AA0DBB1D3B
:104AD0000E94EA26AA81BB810D911C9140E250E020
:104AE000040F151FAA81BB810D931C93A881B98166
:104AF0008C918F5F8C9311F00C9452250C94AC2503
:104B000081E090E0AA81BB818D939C93AC81BD81B3
:104B10004D915C91AA81BB810D911C9104171507E1
:104B200018F011F00C94AC25BB27A0E38C9182FB0C
:104B3000DEF7C29A91E0AA81BB81AD90BC90AFED47
:104B4000B0E0AA0DBB1D0E94EA26AA81BB810E948B
:104B5000CA2511F00C948625C29A83E0481A88274A
:104B6000580A24960895481A8827580A0895480E26
:104B70008827581E08950D911D912D913C9181E03B
:104B8000080F8827181F281F381F3C932E931E9349
:104B90000E930895ED91FC913196FC93EE93089558
:104BA000ED91FC913197FC93EE9308950D911D9139
:104BB0002D913C9101501040204030403C932E9369
:104BC0001E930E93089508D03DD000FC10D0089598
:104BD00003D01ED001F8F9CF0024E89457FF02C09B
:104BE00009D0689400F80BD010F80124089502D081
:104BF00009D00895509540954F5F5F4F0895E89410
:104C000017FF0895009510950F5F1F4F6894089542
:104C1000352F242FE894452B11F468940895512FD3
:104C2000402F0027112780E1440F551F001F111F3F
:104C3000021B130B416018F4020F131F4E7F8A955D
:104C400099F708950F92049F202C312C419F300C2E
:104C5000509F030C022D102D0F900895C8950D92B2
:104C600031960020D9F708958F938D918823E9F725
:104C700011978F91089581E05F9B88270895882779
:104C80005F9B089500C05F9BFECF8CB10895A8E69E
:104C9000B7E08D91882311F011D0FBCF08950E94C9
:104CA0001D27802D11F00AD0FACF08958D9106D0DE
:104CB0003A95E1F708958DE001D08AE05D9BFECF43
:104CC0008CB9089588EE93E0A3D03197D9F7089571
:104CD00050D00AD000FC05D008954BD020D001F868
:104CE000F9CF52D05AD00895842F952FA62FB72FE1
:104CF0004427552766277727F1E2889409C020F4D6
:104D0000480F591F6A1F7B1F7695679557954795E2
:104D10003795279517950795FA9589F70895842F64
:104D2000952FA62FB72FE894452B462B472B11F430
:104D300068940895402F512F622F732F0027112759
:104D400022273327F0E2440F551F661F771F001FED
:104D5000111F221F331F081B190B2A0B3B0B41602D
:104D600028F4080F191F2A1F3B1F4E7FFA9559F789
:104D700008950024E89477FF02C006D0689400F8F4
:104D800009D010F80124089512D04F5F5F4F6F4F84
:104D90007F4F0895E89437FF08950095109520956A
:104DA00030950F5F1F4F2F4F3F4F689408954095E8
:104DB00050956095709508953197F1F708950E9488
:104DC000FB268C910E94FD268D939A95D1F70E9427
:104DD000FC2608950E94FB268D910E94FD269A953F
:104DE000D9F70E94FC260895BF9ABE98C69ABD9A2C
:104DF00080E58DB90895089508958FB9779BFECF0A
:104E00008FB10895689462F80895E89462F808955F
:104E1000EF93FF93EE27E82BE92B31F0E0EDF7E07D
:104E20003197F1F70197D1F7FF91EF9108955A92D9
:104E30004A92480E8827581E0895C895319600203A
:104E40000895819104D08D938823D9F708958136F0
:104E500018F08B3708F48F7D089580E30EF4839566
:104E600008952E2E3F2E992781918D3209F093952A
:104E70008823D1F79A95E22DF32D112361F00917BC
:104E800018F011F0101B01C0191B28F021F080E26E
:104E90008D931A95E9F780818D3219F48D933196AF
:104EA00004C0222311F08BE28D93091738F031F002
:104EB000091B21F080E38D930A95E9F781918D9389
:104EC0008823E1F7332351F0EA2FFB2F31963395F6
:104ED0008E9182933A95E1F78EE28C930895040FB8
:104EE000151F261F371F0895041B150B260B370BA4
:104EF000089504171507260737070895000F111F97
:104F0000221F331F089500951095209530950F5F4F
:104F10001F4F2F4F3F4F0895019110810EC00191F7
:104F20001191219130810BC00191108117FF05C0B3
:104F30003FEF2FEF04C0008111272227332737FFCF
:104F400003C0E1DF8DE28D93CF93DF93CF92DF92A9
:104F5000EF92AA24BB24CC24DD24EE2440E2CAE054
:104F6000DD2755E093E38881890F87FD9F7083FDDE
:104F7000907F891B89935A95A9F7C0DFAA1CBB1C97
:104F8000CC1CDD1CEE1C4A9551F7E894EFE0FF279E
:104F900082910ED0EB30E0F71EF068948A2D0CD091
:104FA00088278D93EF90DF90CF90DF91CF91089578
:104FB000982F829501D0892F8F70805D26F08033E5
:104FC00009F4089568948D930895002711272227E6
:104FD00033271DD08A3328F4803318F005D015D03C
:104FE000F9CF0EF490CF089580538F93402F512F17
:104FF000622F732F83DF82DF72DF80DF8F9199272B
:10500000080F191F291F391F08958D910895E894DD
:10501000FCDF8032E9F38B32D9F38930C9F38D326A
:1050200011F46894F2CF089588278D9308958191A3
:105030008D938823E1F7089509919191992351F077
:105040008A95D9F7319781918D930A9519F0882324
:10505000D1F70895E9CFE199FECFEEBBFFBB3196C2
:10506000089591E001C092E07B3751F47FB7F89446
:10507000F2DF8D918DBBE29AE19A9A95C9F77FBFD5
:105080007727089591E001C092E0E5DFE09A8DB3C3
:105090008D939A95D1F70895FF93881BF9E0001F2F
:1050A000FA9511F4FF910895881F841B18F4840F5A
:1050B0008894F5CF0894F3CF8FEF83959D91992332
:1050C000E1F70895689401C0E894AF93BF938D9180
:1050D00016F0919103C00E941D27902D891718F09A
:1050E00011F48823A1F7BF91AF9108955069636FC0
:1050F0004A62205265616C6974792D53797320344A
:105100002E363100454570726F6D20002C004B45E6
:10511000593136204F4E00004B45593136204F460D
:1051200046004D4D4320696E6974200072657472AB
:1051300079202E2E2E0044535020696E6974200071
:105140004F0021005A003100320033003400350096
:10515000360037003800390030005900570052003F
:1051600048004E00500042005800440045005600E0
:105170004D005300540049004C0020004420000022
:105180002E006F6B00004E6F2063617264004261FD
:105190006420636172640000506172746974696FA5
:1051A0006E2074797065203A0000506172746974E1
:1051B000696F6E2073746172743A00005365637492
:1051C0002F636C757374657220203A00526F6F7490
:1051D000203A000052656164206572726F7220315E
:1051E000000052656164206572726F722032206F18
:1051F0006E20736563746F723A20000052656164BB
:10520000206572726F722033000052656164206500
:1052100072726F7220340000526561642065727290
:105220006F7220350000526561642074696D656F8E
:045230007574000091
:00000001FF
